:040000000A1678283C
:08000800FF00030EF8000A0ED0
:0C001000F900040EFA008A110A160729F4
:10002000A308031D14280800F93000000000000098
:1000300000000000000000000000000000000000C0
:1000400000000000000000000000FF3E031D152816
:1000500000000000000000000000000000000000A0
:100060000000000000000000000000000000000090
:100070000000A30B1428080000000000E00B3C283F
:1000800008005F08E400E3010310E40DE30DE40D54
:10009000E30DE4070318E30AE4070318E30A5A3000
:1000A000E4070318E30A003063078A006008E300EE
:1000B0006408820000308A000030E40082307B282F
:1000C00000308A000030E40094307B2800308A0041
:1000D0000030E400D9307B2800308A000130E40091
:1000E0000A307B2800308A000130E40030307B2861
:1000F0000130E4006130E3070318E40A64088A0071
:1001000063088200273421342234243425342734F0
:1001100029342B342E343134343438343C344134A3
:1001200047344E34573400342034203420343034B3
:1001300020343434353430342034353430343034B1
:10014000203435343534303420343634303430349F
:10015000203436343534303420343734303430348D
:10016000203437343534303420343834303430347B
:100170002034383435343034203439343034303469
:100180002034393435343034313430343034303450
:100190003134303435343034313431343034303437
:1001A0003134313435343034313432343034303425
:1001B0000034493461346D346234693463342D342D
:1001C0004134493461346D346234693463342D34DC
:1001D000423455346C34743469346D34613474345D
:1001E000203442345534473420346B346534793408
:1001F000203453347434723461346934673468346D
:1002000074344F344634463420342034203420347F
:100210002034003453347534703470346C34793491
:10022000543475346E346534203420344B346534A2
:1002300079346534723420344F3466346634733420
:100240006534743454346F346E346534203420345F
:10025000443465346C3461347934203400340034EF
:100260002034203453343034203420345334313467
:100270002034203453343234203420345334333453
:10028000203420345334343420342034533435343F
:10029000203420345334363420342034533437342B
:1002A0002034203453343834203420345334393417
:1002B00039342B343134303439342B343234303413
:1002C0000034053404340334013400340034FA308B
:1002D00083120317A3001020FA30A3001020FA3075
:1002E000A3001020FA30A300102083160313CB0BB9
:1002F00067290800BE08031D7E2908000930000098
:10030000FF3E031D7F2900000000BE0B7E29080070
:10031000231C8D29031306168F29031306120317B6
:10032000A31C952903138616972903138612031716
:10033000231D9D29031306179F2903130613031773
:10034000A31DA52903138617A729031386130715D1
:1003500007110800210E0F39A2002208A3008821EE
:1003600003172108A300882102300317A3001020DF
:100370000800B801B901B501B601B701371A080084
:100380000310B50DB60DAF0DB00DB80DB90D320897
:100390003902031DCD2931083802031CD629310842
:1003A000B8023208031CB903B9023514B70ABE29D2
:1003B000B701B801B7190800361CE0293508B8079D
:1003C000B60C0310B50DB70ADA29B701B801BA01A6
:1003D000BB01B901391A08000310BA0DBB0DB30DEA
:1003E000B40DB70DB80D2E083802031DF9292D08DC
:1003F0003702031C022A2D08B7022E08031CB8037B
:10040000B8023A14B90AEA29A60183160313EF01C8
:1004100083138312031722188317210883160313EB
:100420006F078400EF0A000883120317A500A508D0
:1004300003192F2B2508253A031D2E2A8313221872
:1004400083172108831603136F078400EF0A00083F
:1004500083120317A500253A031D382A8313201899
:1004600083171F0826078400A60A25088000082A8B
:10047000A80129102030A700A50803192F2B250853
:10048000303A0319502A2508203A0319532A25081F
:100490002B3A0319562A25082D3A0319592A682A96
:1004A0003030A7005A2A2030A8005A2A2B30A80042
:1004B0005A2A291483132218831721088316031339
:1004C0006F078400EF0A000883120317A5003C2A77
:1004D000AA012508303C03188D2A2508393C031C45
:1004E0008D2A2A08B5000A30B600D8213808AA009B
:1004F0002508AA073030AA0283132218831721087F
:10050000831603136F078400EF0A00088312031792
:10051000A500A50803192F2B692A25086F3A03198E
:10052000A22A2508643A0319A52A2508753A031951
:10053000AE2A2508583A0319B12A2508623A031948
:10054000B42A2F2B0830AD00B62AA41FAE2A2D30B6
:10055000A800A309A409A30A0319A40A0A30AD003C
:10056000B62A1030AD00B62A0230AD00AB01230828
:10057000B5002408B600AB0A3508B3003608B4004D
:100580002D08AD00AE01E5213A08B5003B08B600E4
:10059000B508031DBB2AB608031DBB2AA808031D06
:1005A000AB0AAC012A08003C0318E02A2B082A02F7
:1005B0000318DC2A2A08AB002B082A02AC00E32A25
:1005C0002B08AA00AC01AC08031929102A08A607B9
:1005D000A9102918A914AB08031DF12AAC080319A6
:1005E0002C2BA603A91CFA2A2708A500AC03031983
:1005F000A910232BAB03031D032BA8080319032BFE
:100600002808A500202B2308AF002408B0002D08DF
:10061000B100B201B9213808A5002508093C03182A
:10062000142B3730A507162B3030A5072308B3004D
:100630002408B400AE01E5213A08A3003B08A40059
:10064000AB080319A9148313201883171F08260762
:10065000840025088000EB2A2A08A607082A8313AD
:10066000201883171F082607840000308000080028
:10067000831205128316630883120317A100AA21AF
:10068000080083160313EF01831205168313031763
:10069000201883171F08831603136F078400800830
:1006A00003190800831383120317201883171F08E8
:1006B000831603136F078400EF0A000883120317E1
:1006C000A100AA21462B5F08E0000310E00D0310F3
:1006D000E00D0310E00DC130600483129F00143060
:1006E0008316E0003C2083121F151F19752B1E086E
:1006F0008316E000E1016008A2006108A30022085F
:10070000A300A2011E08A20483129F010800013069
:1007100083120317A00010309F00831603135F0895
:1007200083120317A10083160313600883120317B3
:10073000A20083160313660883120317A30083160F
:100740000313670883120317A40004220130A000DA
:1007500010309F00412308006203031DB42B610881
:10076000C03EE300382308006108803EE3003823E0
:100770000800831203179701980199019A019301C8
:1007800094019501960183160313EF01EF1A0800F7
:10079000031083120317930D940D950D960D831678
:1007A0000313DF0DE00DE10DE20D83120317970D2A
:1007B000980D990D9A0D831603136608831203177B
:1007C0001A02031DF92B83160313650883120317FE
:1007D0001902031DF92B83160313640883120317F0
:1007E0001802031DF92B83160313630883120317E2
:1007F0001702031C252C83160313630883120317A7
:1008000097028316031364080318092C640F092C3C
:100810000C2C831203179802831603136508031820
:10082000142C650F142C172C8312031799028316AE
:100830000313660803181F2C660F1F2C222C83122B
:1008400003179A0283120317131483160313EF0A74
:10085000C62BEB01EC01ED01EE01EF01EB1A0800F4
:10086000631C402C5F08EC0760080318600FED075D
:1008700061080318610FEE0762080318620FEF07A3
:100880000310E60CE50CE40CE30C0310DF0DE00DA7
:10089000E10DE20DEB0A2E2C831203179501960150
:1008A0009701980199019A019B019C0183160313FA
:1008B000EF01EF1A0800031083120317990D9A0D28
:1008C0009B0D9C0D83160313E70DE80DE90DEA0D52
:1008D00083120317950D960D970D980D831603132C
:1008E0006E08831203171802031D8C2C8316031342
:1008F0006D08831203171702031D8C2C8316031334
:100900006C08831203171602031D8C2C8316031325
:100910006B08831203171502031CB82C83160313EC
:100920006B08831203179502831603136C080318D0
:100930009C2C6C0F9C2C9F2C831203179602831601
:1009400003136D080318A72C6D0FA72CAA2C831274
:1009500003179702831603136E080318B22C6E0F49
:10096000B22CB52C831203179802831203171914A3
:1009700083160313EF0A592C8316031325138312CE
:10098000071308005708831203179F0083160313E9
:10099000580883120317A0004123080003178C187E
:1009A000CE2C03135708831203178D0083160313ED
:1009B0005808831203178C0083168C130C158B13A5
:1009C00055308D00AA308D008C140C118B17080047
:1009D0005708831203178D0083168C130C1483128F
:1009E0000C0883160313D8000800DD01E301E401BD
:1009F0005708E100E201DD190800581C052D6108C7
:100A0000E3070318E40A6208E407D80C0310E10DB9
:100A1000E20DDD0AFB2CD901DA01DB01DC01DD018D
:100A2000D21F1E2DD917D109D209D309D409D10A51
:100A30000319D20A0319D30A0319D40AD91A3C2D6F
:100A4000511C302D4D08DA074E0803184E0FDB07F6
:100A50004F0803184F0FDC0750080318500FDD072D
:100A60000310D40CD30CD20CD10C0310CD0DCE0D31
:100A7000CF0DD00DD90A1E2DD91F0800DA09DB09C8
:100A8000DC09DD09DA0A0319DB0A0319DC0A031998
:100A9000DD0A0800C501C801C9013F08C6004008B9
:100AA000C700451A0800411C5B2D4608C8074708C7
:100AB0000318470FC9070310C20CC10C0310C60D61
:100AC000C70DC50A512D8316031325178312071767
:100AD000080083160313BB01A51183128713BC24DE
:100AE00083162F1C752D8312071683162F180800E6
:100AF000831207120800D70803199F2D0130E30065
:100B00003823013083160313E100E201AC23031301
:100B100005168316DE0106305E0203189F2D380885
:100B2000DF005E08003EE000412083120317A100B1
:100B30008A110A12AA2183160313DE0A8B2D0130B3
:100B4000DF00632383162208D8002308D900DA01C6
:100B5000DB015808DF005908E0005A08E1005B0893
:100B6000E2009330E3000730E400E501E6012924C8
:100B70006C08E7006D08E8006E08E9006F08EA00FD
:100B80006708D8006808D9006908DA006A08DB003D
:100B90005808E7005908E8005A08E9005B08EA002D
:100BA000E830EB000330EC00ED01EE014C24831241
:100BB0000317190883160313A200831203171A08D8
:100BC00083160313A3005808DF005908E0005A08F1
:100BD000E1005B08E200E830E3000330E400E501F7
:100BE000E601B92383120317170883160313DC00E9
:100BF00083120317180883160313DD0001305D020A
:100C0000031D042EF4305C02031C0A2EA20A031DED
:100C10000A2EA30A0230E1000130E200AC23831661
:100C20000313220883120317B30083160313230848
:100C300083120317B4006430AD00AE01E5213A0819
:100C400083160313DC00831203173B088316031378
:100C5000DD002530E1003230E2006430E300E401E1
:100C60000030E000E130DF005C08E6005D08E700EE
:100C700087232E30E1002530E2006430E300563057
:100C8000E400E5010030E000E130DF0022088312DB
:100C90000317AF0083160313230883120317B00052
:100CA0006430B100B201B9213808B3003908B4008A
:100CB0000A30AD00AE01E5213A0883160313E600C1
:100CC000831203173B0883160313E70087230800EA
:100CD000AD08031D0800D80183128718732E013058
:100CE0008316D800882E8719792E03308316D800F2
:100CF000882E8316571C882E83128619832E053062
:100D00008316D800882E0619882E04308316D80042
:100D10008316AB080319AC2ED808031D9F2E2C0890
:100D2000093C0318AC2E2519AC2E2B08AD00AD08DC
:100D30000319AC2E2C08503C031CAD17AC2E5808E0
:100D40002B06031DAC2E2C08503C0318AC2E803013
:100D50002B04AD00AC0125155808AB00AB08031DF2
:100D60000800AC0125110800831603132D08D700D5
:100D7000AD015708D800080083160313B708031DF8
:100D8000BC2E3230B70008003E08C2003F08C30046
:100D90004108003C0318D82E8313431883174208D8
:100DA0008400C20A0319C30A40088000C103C82E88
:100DB0003E08C4003F08C50008000F308312031727
:100DC000A3001020831603130512871307110612C0
:100DD0008612061386138312051203300317A3002D
:100DE000882105300317A3001020031307150711EE
:100DF0000F308316BE007A218312071507110530C4
:100E00000317A300102003130612071507110F3054
:100E10008316BE007A21A517283083120317A1007C
:100E2000AA210830A100AA210C30A100AA21063075
:100E3000A100AA210130A100AA218030A100AA218D
:100E4000031305160800023083160313DF00632323
:100E500000308316C2002030C50039088312031702
:100E6000B5001830B600D821380883160313C30024
:100E7000C4014408C30745084307C1000318C20A58
:100E80000B30C000C00803195B2F8313421883176F
:100E9000410884004008C3000310430D8407230861
:100EA000840A0002031D572F220884030002031C3A
:100EB0005B2FC003422F0430E1000130E200AC237D
:100EC000031305168316BF0104303F020318080000
:100ED0003C08DF004008C500C6010310C50DC60D63
:100EE0000310C50DC60D3F084507E00041208312E1
:100EF0000317A1008A110A12AA2183160313BF0A3D
:100F0000642F83160313E1010130E200AC23831642
:100F10000313AF08031D992F4330BF005730C000A3
:100F20002030C100C2010030D800BF30D700C22439
:100F300008005330BF00C0004230C100C201003081
:100F4000D800BF30D700C224080083160313251C25
:100F50000800C001C101C201C301BF0104303F024A
:100F60000318E02F831283136830840083163F0830
:100F7000CD00CD0D4D0DFC3984070008CE00840A4C
:100F80000008CF00840A0008D000840A0008D100BD
:100F90004008CE0741080318410FCF074208031845
:100FA000420FD00743080318430FD1074E08C00073
:100FB0004F08C1005008C2005108C300BF0AAE2F3D
:100FC0000310C30CC20CC10CC00C0310C30CC20C28
:100FD000C10CC00C4008E7004108E8004208E900E5
:100FE0004308EA000310E70DE80DE90DEA0D0310D0
:100FF000E70DE80DE90DEA0D0310E70DE80DE90D29
:10100000EA0D0310E70DE80DE90DEA0D0310E70DF9
:10101000E80DE90DEA0D1030EB002730EC00ED0192
:10102000EE014C2483120317190883160313CD0015
:10103000831203171A0883160313CE0083120317B3
:101040001B0883160313CF00831203171C08831693
:101050000313D0004D08C0024E08031C4E0FC102FE
:101060004F08031C4F0FC2025008031C500FC3024D
:10107000A0088A15031D3F28A1080319B7284008B6
:10108000C4004108C5004208C6004308C7008312D7
:101090000618702883162008D1002108D200D30139
:1010A000D4016430CD00CE01CF01D0018A110B25CF
:1010B0005A08D5005B08D6005C08D7005D08D80048
:1010C0005508C40756080318560FC50757080318D4
:1010D000570FC60758080318580FC7078A159428D2
:1010E00083162008D1002108D200D301D401643036
:1010F000CD00CE01CF01D0018A110B255A08D500B1
:101100005B08D6005C08D7005D08D8005508C4020B
:101110005608031C560FC5025708031C570FC6027A
:101120005808031C580FC7028A15C71FAF28440967
:10113000CD004509CE004609CF004709D000CD0FAC
:10114000A628CE0FA628CF0FA628D00A4D08C0008B
:101150004E08C1004F08C2005008C300B728440819
:10116000C0004508C1004608C2004708C300E101AD
:10117000E2018A11AC230030A000C8309F00253066
:101180009000323091006430920093010130A2004F
:101190001030A100831603134008E7004108E8005F
:1011A0004208E9004308EA00A030EB008630EC007A
:1011B0000130ED000030EE004C24831203171908B3
:1011C000A3001A08A4000422003083160313D800D9
:1011D000C830D700C2242E30CF00D0010030D80054
:1011E000CF30D700C2244008DF004108E0004208A9
:1011F000E1004308E200A030E3008630E400013063
:10120000E5000030E600B9238312031717088316A0
:101210000313C00083120317180883160313C100B9
:1012200083120317190883160313C20083120317CE
:101230001A0883160313C300003083120317A0009B
:10124000C8309F002530900030309100333092003C
:101250006430930094010130A2001030A100831685
:1012600003134008E7004108E8004208E90043088A
:10127000EA006430EB00EC01ED01EE014C24831236
:1012800003171908A3001A08A400042200308316CB
:101290000313D800C830D700C2242C30CF00D001AF
:1012A0000030D800CF30D700C2240030831203179B
:1012B000A000C8309F00253090006430910092015A
:1012C0000130A2001030A100831603134008DF0094
:1012D0004108E0004208E1004308E2006430E30016
:1012E000E401E501E601B923831203171708831609
:1012F0000313E70083120317180883160313E8008B
:1013000083120317190883160313E90083120317C6
:101310001A0883160313EA000A30EB00EC01ED0112
:10132000EE014C24831203171908A3001A08A40025
:101330000422003083160313D800C830D700C2241B
:101340002510080083160313DF018A116323193067
:101350008316BF00C0012208C1002308C2004A252D
:10136000480883120317B300831603134908831236
:101370000317B4000030AD000430AE00E5213A0898
:1013800083160313C300831203173B08831603134A
:10139000C4004308283CB300143033028A150318F4
:1013A000D4291430B30008003308323C0318080075
:1013B0003230B30008008316031357108A116826D1
:1013C000AD0803190800B4265808C000BC26323006
:1013D000AE004003031908004008023A0319080050
:1013E0004008833A8A150319FE294008033A031975
:1013F0003B2A4008813A0319512A08000130E300D2
:101400008A113823203083160313D900E0003330CB
:10141000DA003630DC004130DD004530DE00463099
:10142000DF005A30DB00E1010030D800D930D700AE
:10143000C224E1010130E200AC2320308316031303
:10144000DB002E30DD00DF003030E0003130DE0028
:101450004630D9004B30DA007630DC00E101003054
:10146000D800D930D700C2240330CB006721013027
:10147000E30038230800AF08031D432A0130AF0002
:1014800083120716462AAF018312071283162F1CF8
:101490004B2A8312071683162F180800831207128F
:1014A0000800BF01C101013083160313E3008A1154
:1014B0003823253083160313D9003130DA00643025
:1014C000DB002E30DC00DD010030E000D930DF0031
:1014D0003F08E600E701E60A0319E70A87238312BB
:1014E00005168316C001063040028A150318932A98
:1014F0003808DF000630D7003F08D8008A11F524ED
:101500006308DB006408DC0040085B07E000412062
:1015100083120317A1008A110A12AA21831603134A
:10152000C00A8A15732AE1010130E2008A11AC2356
:10153000031305168316BF088A150319B32A3F083B
:10154000023A0319B82A3F08053A0319DB2A3F0378
:101550000319002B3F08033A0319032B3F08043AF1
:101560000319902BBC2BD7018A117B258A15BC2B24
:10157000C001083040020318BC2B3108DF003008DE
:10158000D700D8010310D70DD80D0310D70DD80DF3
:101590000310D70DD80D40085707E0008A114120ED
:1015A00083120317A1008A110A12AA2183160313BA
:1015B000C00A8A15B92A003083120317A000C2306E
:1015C0009F00253083160313D7006430D800D9015B
:1015D000003083120317A200D730A1008316031333
:1015E000350883120317A300A4018A1104220030D6
:1015F00083160313D800C230D700C2248A15BC2B2F
:101600005A30BB00BC2B003083120317A000C2303D
:101610009F00253083160313D7003030D8003230B6
:10162000D9006430DA00DB01003083120317A20016
:10163000D730A10083160313200883120317B300C9
:1016400083160313210883120317B400E830AD009A
:101650000330AE008A11E5213A08A3003B08A4003C
:101660000422003083160313D800C230D700C224EE
:101670002E30D900DA010030D800D930D700C2248A
:10168000003083120317A000C2309F00253083165C
:101690000313D7003030D8003330D9006430DA007B
:1016A000DB01003083120317A200D730A10083169C
:1016B0000313200883120317AF00831603132108B6
:1016C00083120317B000E830B1000330B200B92133
:1016D0003808A3003908A40004220030831603133D
:1016E000D800C230D700C2242C30D9003030DA0004
:1016F000DB010030D800D930D700C2243D08DF001C
:101700004108E0004120E1000130E2008A110A12A4
:10171000AC230F3083160313E30038238A15BC2B48
:10172000C001043040020318B02B2808DF0029084C
:10173000D700D8010310D70DD80D0310D70DD80D41
:1017400040085707E0008A11412083120317A100C7
:101750008A110A12AA2183160313C00A8A15912B33
:10176000A9080319BC2B483083120317A1008A1162
:10177000AA217A30A100AA2183160313AD088A1585
:10178000031DCD2BAE08031DC82B3F03031D2D2DBC
:1017900057148A1168268A15BC2B8A11B42658085A
:1017A000C000BC263230AE00692583164008813A5D
:1017B0008A150319F22B4008043A0319FD2B40083F
:1017C000843A0319FD2B4008053A0319982C400868
:1017D000853A0319982C400303192D2D3F03031953
:1017E0002D2D532ABF0A06303F020318BF010C30CB
:1017F000E3008A1138238A15532A3F08043A031953
:10180000112C3F08023A0319192C3F08053A031915
:101810001F2C3F0303192D2D3F08033A0319212CD8
:10182000532A103029020318172CA90AB32CA90136
:10183000B32CB00A3008053C031CB001532AB50A8A
:10184000532A4008843A031D3F2C043041020318F8
:101850002B2CC10A2C2CC1013D08DF004108E000FF
:101860008A114120E1000130E2008A110A12AC2302
:101870000F3083160313E30038238A15532A4008D8
:10188000043A031D532AC108031D512CA008031D4F
:101890004C2CA1080319512CA0080319A103A00383
:1018A000532A4103031D612C00302102031D5A2CD1
:1018B0000A302002031C612C0A30A002031CA10381
:1018C000532A4108023A031D722C00302102031DE5
:1018D0006B2C64302002031C722C6430A002031CA9
:1018E000A103532A4108033A031D852C033021022A
:1018F000031D7C2CE8302002031C852CE830A0025C
:101900000330031CA103A102532A4108043A031D1A
:10191000532A27302102031D8F2C10302002031C74
:10192000532A1030A0022730031CA103A102532A1E
:101930003F08043A0319AC2C3F08023A0319C32CA0
:101940003F08053A0319CB2C3F0303192D2D3F08FF
:10195000033A0319CD2C532AA9080319B12CA90362
:10196000B32C1030A900A9080319B82C2516B92CDE
:1019700025122708DF002908E0008A114120AA006B
:101980008A150A12532AB0080319C82CB003532A27
:101990000530B000532AB503532A4008853A031D89
:1019A000EB2CC1080319D62CC103D82C0430C1007C
:1019B0003D08DF004108E0008A114120E1000130CC
:1019C000E2008A110A12AC230F3083160313E300DE
:1019D00038238A15532A4008053A031D532AC108A3
:1019E000031DF62CA00A0319A10A532A4103031D63
:1019F000FE2C0A30A0070318A10A532A4108023A14
:101A0000031D072D6430A0070318A10A532A4108BB
:101A1000033A031D1A2D4A302102031D112D3730C0
:101A2000200203181A2DE830A00703300318A10A7A
:101A3000A107532A4108043A031D532A27302102E3
:101A4000031D242D0F3020020318532A1030A00745
:101A500027300318A10AA107532A3F08043A0319A3
:101A60003E2D3F08023A03194F2D3F08033A031950
:101A7000602D3F08053A0319CC2DDB2D0D30D70022
:101A80008A11E824290858068A150319DB2D0D3020
:101A9000D7002908D8008A11CE248A15DB2D0A30F8
:101AA000D7008A11E824300858068A150319DB2D5F
:101AB0000A30D7003008D8008A11CE248A15DB2DD1
:101AC0002008CF002108D000D101D2010C30D7006E
:101AD0008A11E8245808CB00CC01CD01CE010310B7
:101AE000CB0DCC0DCD0DCE0D0310CB0DCC0DCD0DF2
:101AF000CE0D0310CB0DCC0DCD0DCE0D0310CB0DA7
:101B0000CC0DCD0DCE0D0310CB0DCC0DCD0DCE0DCE
:101B10000310CB0DCC0DCD0DCE0D0310CB0DCC0D88
:101B2000CD0DCE0D0310CB0DCC0DCD0DCE0D0B304C
:101B3000D700E8245808D300D401D501D6014B08BA
:101B4000D3074C0803184C0FD4074D0803184D0F4A
:101B5000D5074E0803184E0FD60753084F028A15B3
:101B6000031DBE2D54085002031DBE2D5508510201
:101B7000031DBE2D560852020319DB2D0C30D70071
:101B80002108D8008A11CE240B300313D700200877
:101B9000D800CE248A15DB2D0E30D7008A11E82418
:101BA000580835068A150319DB2D0E30D700350885
:101BB000D8008A11CE248A1169250C308316E300DF
:101BC0003823013083160313E300382308008316FB
:101BD0000313AF080319F52D83128619F22D8A110C
:101BE000632508008A11BC24080005303002031860
:101BF0000800B2080319192E32080B3A0319382EBF
:101C000032080C3A0319462E3208153A0319622E8F
:101C100032081F3A0319792E3208163A0319B12EE9
:101C20003208213A0319C52E3208063A0319012F4A
:101C3000B20183128619262E0B308316B2008A1148
:101C4000632583163408B6008A15382E83163008AB
:101C5000043A031908008312061908000C30831691
:101C6000B2008A11632583163408B6008A15462E01
:101C7000B608031D0800251FFC2E3308B6001530DA
:101C8000B200251AA515831287170800B608031D90
:101C90000800251FFC2E033083120317B50083169E
:101CA0000313330883120317B6008A11D8213808AA
:101CB00083160313B6001630B200251AA515831239
:101CC000871708003008043A031D6E2E8312861D04
:101CD00008008316A51183128713FC2EB608031D76
:101CE0000800A5118312871383163308B6001F302E
:101CF000B200B608031D08003008023A031D8F2EFB
:101D0000831206198C2E86198C2E8316A51E8A2EF8
:101D1000A516DB2EA5168F2E8316A512DB2E831299
:101D20000619A52E03300317B500831603133308D5
:101D300083120317B6008A11D821380883160313BB
:101D4000B6001630B2008A15AC2E8619FC2E83160A
:101D50003308B6001530B200251AA515831287176F
:101D600008003008033A031DB92E8312061D08002F
:101D7000BC2EB608031D08008316A5118312871315
:101D800083163308B6002130B200B608031D0800E0
:101D90003008023A031DDB2E83120619D82E86194D
:101DA000D82E8316A51ED62EA5168F2EA516DB2E91
:101DB0008316A5128F2E83128619E42E83163308FC
:101DC000B6001530B200F72E0619FC2E03300317AB
:101DD000B50083160313330883120317B6008A1164
:101DE000D821380883160313B6001630B200251A1E
:101DF000A51583128717080083163508B60006302C
:101E0000B200831286190A2F83163308B6001530E4
:101E1000B200302F0619252F83163008043A031913
:101E2000252F033083120317B500831603133308DD
:101E300083120317B6008A11D821380883160313BA
:101E4000B6001630B2008A15302F8316B608031D6F
:101E50000800B201A511831287138A11BC2408005F
:101E6000251AA5158312871708008B13EF308316E8
:101E70000313850080309F00FF3083128500831696
:101E800086008312860183168113071387130712B6
:101E90008A11BC248713831687148715DD268316C1
:101EA000BB01FB01FC01A5118B128312810183167A
:101EB000811281110111811401108B168B16A6015C
:101EC00083121211910159309200D0308316920082
:101ED0008C1483121215063090008F018E010C10A5
:101EE00083160C140B178B170D30D700E8245808F5
:101EF000A9002908103C8A150318862F0530A9006F
:101F00000D30D7002908D8008A11CE240313871278
:101F1000A511A9088A1503198F2F2516902F2512B0
:101F20002708DF002908E0008A114120AA00FD01EE
:101F3000FE0125100030BF006830BE00C001103027
:101F4000C1008A110A12C4260C30D700E8245808B0
:101F5000C200C301C401C5010310C20DC30DC40DED
:101F6000C50D0310C20DC30DC40DC50D0310C20D68
:101F7000C30DC40DC50D0310C20DC30DC40DC50D99
:101F80000310C20DC30DC40DC50D0310C20DC30D4A
:101F9000C40DC50D0310C20DC30DC40DC50D031036
:101FA000C20DC30DC40DC50D0B30D700E824580871
:101FB000C600C701C001C1014208C6074308031893
:101FC000430FC7074608A0004708A100B9018A15BA
:101FD000A2210A30D7008A11E8245808B00030083E
:101FE000053C8A150318FB2FB0010A30D7003008D2
:101FF000D8008A11CE24831203138A110A160619F7
:10200000042804308316B0008316AF018312071230
:102010008316B201A5120A12BC240E308316D70013
:10202000E8245808B5000530B400AB01AD01251116
:10203000AC010130E3003823203083160313C000C5
:10204000C7002130C6004830C1006530C2006C3086
:10205000C300C4006F30C500C8010030D800C030D4
:10206000D700C224E1010130E200AC232030831606
:102070000313C000C100C200C500C600C7004D3038
:10208000C4004F30C300C8010030D800C030D700B2
:10209000C2240230CB006721BC26643083120317B0
:1020A000A3001020BC26643083120317A300102065
:1020B000BC260130D7007B250230CB0067210130E0
:1020C000E30038238A150A12A221E7258316BE01F0
:1020D000251BBE0ABE088A110A16031D62280A12B1
:1020E000A527812723278A15DB218A110A16622852
:1020F000003083160313A7000130A8000230B1009E
:102100000330B8008312A001A1010D30A200A30189
:102110001A30A400A5013330A600A7016830A8003A
:10212000A901D030AA00AB013830AC000130AD00BD
:10213000A130AE000130AF000930B0000230B10074
:102140007130B2000230B3000730B4000330B50084
:10215000D830B6000330B700B801B9010D30BA006D
:10216000BB011A30BC00BD013330BE00BF01683076
:10217000C000C101D030C200C3013830C4000130FA
:10218000C500A130C6000130C7000930C8000230C8
:10219000C9007130CA000230CB000730CC000330D8
:1021A000CD00D830CE000330CF00D001D1010D30AA
:1021B000D200D3011A30D400D5013330D600D70174
:1021C0006830D800D901D030DA00DB013830DC00CB
:1021D0000130DD00A130DE000130DF000930E00019
:1021E0000230E1007130E2000230E3000730E40029
:1021F0000330E500D830E6000330E70004308316F2
:10220000BC000530BD00A5138A150A12352F8312B4
:1022100003138C1CDE298C108316A60A6430260258
:102220000318A60125189D29A608031D212983123C
:10223000121191018F018E01FD01FE011215101482
:102240009D292608323A031D9D29831210108316FA
:10225000A40A7D0883120317C7007E08C800BF01C7
:10226000C001C501C60103130F080317C100C20155
:10227000C301C4010310C10DC20DC30DC40D031071
:10228000C10DC20DC30DC40D0310C10DC20DC30D90
:10229000C40D0310C10DC20DC30DC40D0310C10D3B
:1022A000C20DC30DC40D0310C10DC20DC30DC40D6D
:1022B0000310C10DC20DC30DC40D0310C10DC20D1D
:1022C000C30DC40D41084504CD0042084604CE00AC
:1022D00043084704CF0044084804D00003130E0805
:1022E0000317C900CA01CB01CC0149084D04D10034
:1022F0004A084E04D2004B084F04D3004C08500447
:10230000D40003138313683084000330831624053C
:1023100083120317BC00BC0D3C0DFC398407510827
:1023200080005208840A80005308840A8000540800
:10233000840A80008316031325148316B608031D30
:10234000B603BA0A3A08043C0318C529BA012C0896
:10235000F03C003C2C020318F03A0319B129AC0AF6
:10236000B229AC01BB080319C529BB03BB08031D77
:10237000C529831207128316251EBF29A5158312AE
:10238000871783162517831207178316B7080319B3
:10239000D029B703B7080319CF29A515D029A5114E
:1023A000FB0A0319FC0A32307B0603197C08031D63
:1023B000DE29FB01FC01AE08031DAE0383120C1CD9
:1023C000E5290C10FD0A0319FE0A0B1DFD290B114E
:1023D00083162A08831281008316A51DF329250878
:1023E000023AA500F429A510A51CF8298312871626
:1023F0008316A518FD29831287127A0E8400790EA0
:0C2400008A00780E8300FF0E7F0E09009A
:02400E007A3FF7
:00000001FF
